:020000040800F2
:1000000000100020D51B000885040008910400089A
:1000100000000000000000000000000000000000E0
:10002000000000000000000000000000950400082F
:100030000000000000000000A1040008AD0400085A
:10004000211C000800000000211C0008211C0008E1
:10005000211C0008211C0008211C0008211C00088C
:10006000000000009B0700084D0D0008211C00083F
:10007000211C0008211C0008211C000800000000B1
:10008000211C00080000000000000000211C0008E6
:1000900000000000C9030008211C0008211C000802
:1000A000000000009D03000800000000410A000855
:1000B0000000000000000000000000000000000040
:1000C00080B582B000AF0200FB1D1A70FB1D1B78CB
:1000D0001A001F231A40044B012191400A001A60A4
:1000E000C046BD4602B080BD00E100E090B583B0DF
:1000F00000AF02003960FB1D1A70FB1D1B787F2BBF
:1001000032D92F4AFB1D1B7819000F230B40083BE7
:100110009B0806339B00D31804331B68FA1D127822
:10012000110003220A40D200FF2191400A00D2436D
:100130001A4011003B689B01FF221A40FB1D1B78EF
:10014000180003230340DB009A401D48FB1D1B7869
:100150001C000F232340083B9B080A4306339B00E7
:10016000C31804331A6027E0164AFB1D1B785BB2E4
:100170009B08C0339B009B58FA1D12781100032284
:100180000A40D200FF2191400A00D2431A401100D8
:100190003B689B01FF221A40FB1D1B7818000323BC
:1001A0000340DB009A400748FB1D1B785BB29B08AD
:1001B0000A43C0339B001A50C046BD4603B090BDF1
:1001C00000ED00E000E100E080B582B000AF7860B3
:1001D0007B685A1E80235B049A4201D3012310E0FE
:1001E0000A4B7A68013A5A6001235B4203211800E6
:1001F000FFF77CFF054B00229A60044B07221A6030
:1002000000231800BD4602B080BDC04610E000E0EB
:1002100080B500AFC046BD4680BD80B500AF534B32
:100220001A68524B802149020A431A60C0464F4B5C
:100230001A6880239B021340F9D04C4B5A684B4BF1
:100240004B490A405A60494B5A68484B8821490338
:100250000A435A60454B1A68444B802149040A43BB
:100260001A60C046414B1A6880239B041340F9D0A2
:100270003E4B5A683D4B02210A435A6000F0B2FFE0
:100280003C4B1B680A21180001F02EFB03001800EC
:10029000FFF79AFF01235B421800FFF711FF0123CC
:1002A0005B4260211800FFF721FF304B5A692F4B4A
:1002B00031490A435A612D4B9A692C4B2F490A4305
:1002C0009A612A4BDA69294B02210A43DA619023A9
:1002D000DB051A689023DB0529490A431A6090233D
:1002E000DB059A689023DB0526490A439A60902330
:1002F000DB0500221A629023DB05882252005A6235
:10030000214A214B12681A60204BC92292001A60C0
:100310001E4BE022D2005A601C4B1A681B4B402136
:100320000A431A601920FFF7CBFE40211920FFF77E
:10033000DDFE174B00225A60154B0122DA60144B88
:100340002F229A62124B134ADA62114B01221A6071
:100350001520FFF7B5FE40211520FFF7C7FE0E4B15
:10036000180000F045F900F0F5FAFEE70010024031
:100370000CF8C3FF0000002051000600015A4200A3
:1003800070A92800808A080000040048003001405D
:1003900000440140E703000040420F0080B500AF79
:1003A000084B9B680222134009D09023DB050822EA
:1003B0009A61044B5A68034B80218A435A60C046B5
:1003C000BD4680BD0030014080B582B000AF284BF3
:1003D0001B690122134047D0254B1A69244B012188
:1003E0008A431A61FB1D00221A70BB1D01221A707C
:1003F00000233B601DE01F4B3A689200D358002B4E
:100400000FD01C4B3A689200D358591E194B3A68CA
:100410009200D150FB1DF91DBA1D097812780A43CC
:100420001A70BA1DBB1D1B78DB1813703B680133B3
:100430003B603B68072BDED90F4B1B68591C0E4AEB
:1004400011600A2B10D10C4B00221A600B4AFB1DC5
:100450001B7813700A4B5A68094B80210A435A6073
:100460009023DB0508229A62C046BD4602B080BDDB
:100470000044014078010020980000200C30014029
:100480000030014080B500AF00BEC046BD4680BD13
:1004900000BEC04680B500AF00BEC046BD4680BDB0
:1004A00080B500AF00BEC046BD4680BD80B500AF80
:1004B0000A4B1B68591C094A11600A2B0AD1074BC9
:1004C00000221A60064B1B685A1C054B1A60054B2C
:1004D00064229A61C046BD4680BDC0469C00002093
:1004E000940000207801002080B582B000AF0200A7
:1004F000FB1D1A70FB1D1B781A001F231A40044BAA
:10050000012191400A001A60C046BD4602B080BD7C
:1005100000E100E090B583B000AF02003960FB1D40
:100520001A70FB1D1B787F2B32D92F4AFB1D1B78BD
:1005300019000F230B40083B9B0806339B00D31880
:1005400004331B68FA1D1278110003220A40D200FE
:10055000FF2191400A00D2431A4011003B689B01E1
:10056000FF221A40FB1D1B78180003230340DB0009
:100570009A401D48FB1D1B781C000F232340083B9D
:100580009B080A4306339B00C31804331A6027E014
:10059000164AFB1D1B785BB29B08C0339B009B581F
:1005A000FA1D1278110003220A40D200FF21914067
:1005B0000A00D2431A4011003B689B01FF221A40F7
:1005C000FB1D1B78180003230340DB009A400748FB
:1005D000FB1D1B785BB29B080A43C0339B001A507B
:1005E000C046BD4603B090BD00ED00E000E100E074
:1005F00080B584B000AF786000F04AF8204B8022CC
:1006000012061A611E4B07225A611D4B1D4ADA6001
:100610001B4B04229A621A4B9A68194B80210906D7
:100620000A439A60C046164B9B68002BFBDB144BB9
:100630009A68134B01210A439A60114B9A68104B38
:1006400004210A439A607B680F4A934206DD7B6867
:10065000FA21180001F0D2F9030000E00623FB6044
:10066000FA6880235B029A4201DB084BFB60FB685F
:1006700019000C2000F05AF8C046BD4604B080BDF9
:100680000024014043080000DC050000FFFF0000DB
:1006900080B500AF0B4B0C4A9A600A4B00221A60DF
:1006A000084B1A68074B09490A431A600920FFF7EB
:1006B0001BFF40210920FFF72DFF00F009F8C0467D
:1006C000BD4680BD08000240402401408205000074
:1006D00080B500AF124B1A68114B01218A431A6092
:1006E000104B1B685A425341DBB21A000D4B1A6083
:1006F0000C4B1A681300DB009B18DB0008331A0050
:10070000094BD218064BDA60054B20225A60044B85
:100710001A68034B01210A431A60C046BD4680BDDA
:100720000800024034010020A000002080B582B003
:1007300000AF78603960154B802212025A64134B67
:10074000C022D201DA61114B802252011A620F4B92
:1007500001221A647B685A1E0C4B9A623B685A1E2F
:100760000A4BDA62094B5A69084B01210A435A6164
:10077000064B80221A60054B1A68044B01210A437C
:100780001A60C046BD4602B080BDC046002C014084
:1007900080B500AFC046BD4680BD80B582B000AF19
:1007A0001A4B1B687B60194B5A68184B01210A438E
:1007B0005A60FFF78DFFFFF7EBFF154B1A88531CAC
:1007C00099B2134B1980134B1B6859424B41DBB252
:1007D000180011490300DB001B18DB00CB1806339F
:1007E0001A800C4B1B685A425341DBB21A001300AB
:1007F000DB009B18DB00084A9B184821180000F01A
:10080000C7FAC046BD4602B080BDC04600000240E7
:100810003001002034010020A000002080B582B00B
:1008200000AF0200FB1D1A70FB1D1B781A001F236E
:100830001A40044B012191400A001A60C046BD468F
:1008400002B080BD00E100E080B582B000AF0200E0
:10085000FB1D1A70FB1D1B781A001F23134005494E
:1008600001229A40130080228B50C046BD4602B040
:1008700080BDC04600E100E090B583B000AF02004B
:100880003960FB1D1A70FB1D1B787F2B32D92F4A54
:10089000FB1D1B7819000F230B40083B9B080633F8
:1008A0009B00D31804331B68FA1D12781100032231
:1008B0000A40D200FF2191400A00D2431A401100A1
:1008C0003B689B01FF221A40FB1D1B781800032385
:1008D0000340DB009A401D48FB1D1B781C000F23C2
:1008E0002340083B9B080A4306339B00C31804338C
:1008F0001A6027E0164AFB1D1B785BB29B08C033C9
:100900009B009B58FA1D1278110003220A40D20066
:10091000FF2191400A00D2431A4011003B689B011D
:10092000FF221A40FB1D1B78180003230340DB0045
:100930009A400748FB1D1B785BB29B080A43C033F3
:100940009B001A50C046BD4603B090BD00ED00E0CC
:1009500000E100E080B582B000AF304B012252428E
:100960001A602E4B00225A602C4B00225A612B4BEE
:1009700000229A61294B012252429A60274B0022A1
:10098000DA60264B00221A6100237B600BE0234AC9
:100990007B6806339B00D3180433012252421A604D
:1009A0007B6801337B607B68072BF0D91C4B1800F8
:1009B00000F04AFB1B4B1C4A9A601A4B92221A60A9
:1009C0001A4B1B4ADA60194B1A4A1A600A20FFF7C1
:1009D00025FF20210A20FFF74FFF174B174A1A6007
:1009E000154BC022DA60144BC02292025A60124B9F
:1009F0009A68114B80210A439A601B20FFF70EFF73
:100A000060211B20FFF738FF0B4B1A680A4B0121AE
:100A10000A431A60C046BD4602B080BD980100205E
:100A2000480100201C0002402838014030000240EC
:100A30000030024042100000003801402C2000002D
:100A400080B586B000AF404BDB693B613B69082253
:100A5000134008D03C4B08221A623C4B1B685A1CBE
:100A60003A4B1A606CE03B692022134000D167E0EA
:100A7000354B9B8C9AB20F217B181A707B181B7810
:100A800033493448202200F0EDFA0300BB60BB6814
:100A9000002B54D0BB68002B05DA2F4B1B685A1C67
:100AA0002D4B1A604CE0BB68022B05D02B4B1B680A
:100AB0005A1C2A4B1A6043E0254B7B607B681B78ED
:100AC000DBB2032B26D030DC012B02D0022B13D05B
:100AD0002BE000237B610BE0214A7B6906339B00FE
:100AE000D3180433012252421A607B6901337B61BF
:100AF0007B69072BF0D921E07B685B78DBB21800BB
:100B000000F09AF8031E16D0144B1B685A1C134BA6
:100B10001A6010E0124B0122DA60124B1B680122AE
:100B200013400AD100F020F807E00C4B1B685A1C58
:100B30000A4B1A6004E0C04602E0C04600E0C0462E
:100B4000BD4606B080BDC046003801403C010020D3
:100B500050010020480100204001002044010020F5
:100B6000980100201C00024080B586B000AF304BD9
:100B7000BB60BB681B69002B08D0BB6800221A61F0
:100B8000BB689B683B6100237B6116E0BB68DB6848
:100B9000002B09D0BB680022DA60BB689B683B6110
:100BA000BB681B687B6108E0BB689B680133072258
:100BB00013403B61BB685B687B61BA683B69063385
:100BC0009B00D31804331B687B607B6801332BD0F8
:100BD0007A687B699A4204DD7A687B69D31AFB6084
:100BE00004E07B6980229200D31AFB60BB687A69BB
:100BF0001A607A69FB68D318DB05DA0DBB685A60A6
:100C0000BB683A699A60BB683C331A007B69D218AA
:100C1000084BDA60074BFA685A60064B1A68054BB6
:100C200001210A431A6000E0C046BD4606B080BDFF
:100C3000980100201C00024080B582B000AF020085
:100C4000FB1D1A70FB1D1B78082B02D916235B4273
:100C50001AE0FB1D1A780E4B9B689A4202D01623AD
:100C60005B4211E0FB1D1B78094A06339B00D31839
:100C70000433012252421A60064B1B6801221340C2
:100C800001D1FFF771FF00231800BD4602B080BDFF
:100C9000980100201C00024080B582B000AF78604F
:100CA0000A00FB1C1A700A20FFF7CEFD7B685A6908
:100CB0007B681B689A4205D10A20FFF7AFFD10231D
:100CC0005B4213E07B685B697A683C21D3185B1850
:100CD000FA1C12781A707B685B690133DB05DA0D48
:100CE0007B685A610A20FFF799FD00231800BD4672
:100CF00002B080BD80B582B000AF0200FB1D1A704B
:100D0000C046FB1D1A78064B11001800FFF7C4FF00
:100D100003001033F5D000231800BD4602B080BD9B
:100D20009801002080B582B000AF0200FB1D1A7050
:100D3000FB1D1A78044B11001800FFF7ADFF0300EC
:100D40001800BD4602B080BD9801002080B500AFFC
:100D50000C4B5A680B4B20210A435A600A4B1A6805
:100D6000094B01218A431A60084BDB68002B03D131
:100D7000064B1B69002B01D0FFF7F6FEC046BD46AF
:100D800080BDC046000002401C00024098010020C7
:100D900090B585B000AF78603960414B9B69404A9F
:100DA00006339B00D31804331B68013307D03D4B37
:100DB0001B685A1C3B4B1A6010235B426CE0384B9B
:100DC0009B69DAB27B681A717B6800225A71364BD4
:100DD000A1229A600423FB6008E07A68FB68D318BC
:100DE0001A78314B1A60FB680133FB60FA683B6884
:100DF0009A42F2D32C4B1B68DA437B68FF211140E7
:100E00000C00197800200140081C211C01431970B6
:100E1000110AFF2001400C00597800200140081CF5
:100E2000211C01435970110CFF2001400C009978DE
:100E300000200140081C211C01439970100EDA7833
:100E400000210A40111C021C0A43DA703A687968D2
:100E5000164B180000F02EF80300BB60BB68002B97
:100E600001D0BB6818E00E4B98690D4B5A690C49CC
:100E7000831D9B00CB1804331A60094B9B69013317
:100E800007221A40064B9A61094B1B680122134046
:100E900001D1FFF769FE00231800BD4605B090BDE3
:100EA000980100203801002000300240250D000884
:100EB0001C00024080B58AB000AFF860B9607A606B
:100EC0007B68FE2B02D901235B424EE000237B624C
:100ED0003CE07B6A002B0FD07B6A013BBA68D318D9
:100EE0001B78002B08D07B6A013BBA68D2182323F9
:100EF000FB1812781A7019E07B6AFB6102E0FB694B
:100F00000133FB61FA697B689A4205D2BA68FB69D2
:100F1000D3181B78002BF2D1FB69DAB27B6ADBB203
:100F2000D31ADAB22323FB1801321A702323FB18D9
:100F30001A78FB681000984703007B617B69002BDF
:100F400001D07B6911E07B6A01337B627A6A7B683E
:100F50009A42BED9FB68002098470300BB61BB6979
:100F6000002B01D0BB6900E000231800BD460AB089
:100F700080BD80B588B000AFF860B9607A603B6032
:100F8000BA6880235B029A4204D23A6880235B02EB
:100F90009A4202D301235B4252E03B68002B02D10C
:100FA00001235B424CE0BA683B689A4202D20123BB
:100FB0005B4245E00123FB617B681B78BB61BB6939
:100FC000002B24D102235B423AE0BB69013BBB61A9
:100FD000BB69002B09D17A68FB69D3181B78BB6108
:100FE0001723FB1800221A7006E07A68FB69D218F2
:100FF0001723FB1812781A70FB69013BFA68D318A3
:101000001722BA1812781A70FB690133FB61FA696A
:101010003B689A4205D27A68FB69D3181B78002B8B
:10102000D3D1FA693B689A4202D102235B4207E0BE
:10103000BB69012B02D003235B4201E0FB69013B4A
:101040001800BD4608B080BD80B582B000AF7860A2
:101050007B6800221A607B6800225A60C046BD4649
:1010600002B080BD80B588B000AFF860B9607A602A
:101070001A00FB1C1A70FB681B68002B0ED1FB1CAE
:101080001B78002B54D0FB1C1A78FB685A60FB6855
:101090001B685A1CFB681A60002350E0FB1C1B787D
:1010A000002B0DD1FB685B68012B39D1FB681B68F5
:1010B000013B7B61FB681800FFF7C6FF7B693EE0E0
:1010C000FB685B685A1EFB685A60FB685B68002B14
:1010D00008D1FB1C1A78FB685A601F23FB180022FA
:1010E0001A7004E01F23FB18FA1C12781A70FB68B0
:1010F0001B68013BBB61BA697B689A4202D3022339
:101100005B421CE0BA68BB69D3181F22BA18127878
:101110001A70FB681B685A1CFB681A6000230EE0FB
:10112000C046FB681800FFF78FFF01235B4206E013
:10113000C046FB681800FFF787FF03235B421800D7
:10114000BD4608B080BD3C1C000800000020940093
:10115000002094000020D4030020000080B500AFE0
:101160001A4B1A68194B01210A431A60174B5A6827
:10117000164B17490A405A60144B1A68134B15490D
:101180000A401A60114B1A68104B13490A401A6042
:101190000E4B5A680D4B11490A405A600B4BDA6AE4
:1011A0000A4B0F218A43DA62084B1A6B074B0C4932
:1011B0000A401A63054B5A6B044B01218A435A6358
:1011C000024B00229A60C046BD4680BD001002401E
:1011D0000CB8FF08FFFFF6FEFFFFFBFFFFFFC0FF9D
:1011E000ECFEFFFF80B584B000AF0023FB6000235E
:1011F000BB6000237B6000233B60314B5B680C22AB
:101200001340FB60FB68082B11D0FB68082B41D80A
:10121000FB68002B03D0FB68042B04D03AE0294B79
:10122000294A1A603AE0274B274A1A6036E0244BD5
:101230005A68F0239B031340BB60214B5A688023FC
:101240005B0213407B60BB689B0C0233BB601C4B92
:10125000DB6A0F22134001333B607A6880235B0214
:101260009A420AD13968184800F03EFB03001A0080
:10127000BB685A43134B1A6010E0B9680A00520168
:10128000521A93019B1ADB005B181B021A000D4BCC
:101290001A6003E00B4B0C4A1A60C046084B5B68AF
:1012A0001B090F221340094AD35CFB60054B1A68E7
:1012B000FB68DA40034B1A60C046BD4604B080BDEF
:1012C000001002400000002000127A00241C0008D8
:1012D00080B500AF044B1A68034B8021C9020A4352
:1012E0001A60C046BD4680BD0010024080B500AF08
:1012F000044B1A68034B04490A401A60C046BD46B5
:1013000080BDC04600100240FFFFFBFF80B500AF6C
:10131000044B1A68034B802149020A431A60C046F5
:10132000BD4680BD0010024080B500AF064B1A6874
:1013300080239B021340054A944663445A4253411A
:10134000DBB21800BD4680BD001002400000FEFF69
:1013500080B500AF044B1A68034B01210A431A60A1
:10136000C046BD4680BDC0460010024080B500AFFB
:10137000054B1B6802221340023B5A425341DBB229
:101380001800BD4680BDC0460010024080B582B046
:1013900000AF7860064B5B68032293431900044B4F
:1013A0007A680A435A60C046BD4602B080BDC04656
:1013B0000010024080B500AF034B5B680C22134065
:1013C0001800BD4680BDC0460010024080B582B006
:1013D00000AF7860064B5B68F02293431900044B22
:1013E0007A680A435A60C046BD4602B080BDC04616
:1013F0000010024080B582B000AF7860064B5B6899
:10140000064A13401900044B7A680A435A60C046E2
:10141000BD4602B080BDC04600100240FFF8FFFF8D
:1014200080B500AF044B1A68034B802149040A437E
:101430001A60C046BD4680BD0010024080B500AFB6
:10144000074B1A6880239B041340FE221206944621
:1014500063445A425341DBB21800BD4680BDC046CA
:101460000010024080B582B000AF786039600E4B4A
:101470005B680E4A134019007A6880235B021A40A9
:101480003B681A43084B0A435A60074BDB6A0F223A
:10149000934319007B680F221A40034B0A43DA6218
:1014A000C046BD4602B080BD00100240FFFFC2FF33
:1014B00080B582B000AF786039603968786800F034
:1014C00013FA03001A00064B013A5A60044B00223B
:1014D0009A60034B05221A60C046BD4602B080BD2B
:1014E00010E000E080B582B000AF7860064B1B686A
:1014F000012293431900044B7A680A431A60C046DC
:10150000BD4602B080BDC0460020024080B500AF9D
:10151000034B1B68012213401800BD4680BDC04626
:101520000020024080B582B000AF7860FA239A00B4
:101530007B6811001800FFF7BBFFC046BD4602B034
:1015400080BD80B584B000AF78600E4B1B68FB6037
:10155000FB687B6801330CD07B6801337B6008E05B
:10156000084B1A6880235B02134002D07B68013B62
:101570007B607B68002BF3D1C046C046BD4604B0FB
:1015800080BDC04610E000E080B582B000AF78605A
:10159000034B7A681A60C046BD4602B080BDC046A3
:1015A0000000002090B585B000AF786039600F234F
:1015B000FB1801221A700023BB6000F0D4F803006E
:1015C000012B28D17B6801225A607B68174A1900D9
:1015D000100000F0ABF80300BB60FFF7C7FE03008C
:1015E000012B07D0FFF7B4FEC046FFF7BFFE030094
:1015F000012BFAD17B681B6819000020FFF732FF2E
:101600000F23FC183A68BB681100180000F0BEF800
:101610000300237003E00F23FB1800221A700F232E
:10162000FB181B781800BD4605B090BD00127A006B
:1016300090B587B000AFF860B9607A603B6017235F
:10164000FB1801221A7000233B6100F08CF80300A4
:10165000012B32D17A68FB681100180000F066F89F
:1016600003003B61FFF760FE0300012B0FD0BB6856
:10167000012B02D1FFF72CFE01E0FFF737FEFFF749
:1016800045FEC046FFF750FE0300012BFAD17B68F0
:101690005B68802252021A437B681B6819001000A5
:1016A000FFF7E0FE1723FC183A683B6911001800A9
:1016B00000F06CF80300237003E01723FB180022EE
:1016C0001A701723FB181B781800BD4607B090BD91
:1016D00080B584B000AF78600F217B1801221A70AA
:1016E0000023BB607B68002B03D17B1800221A709B
:1016F00013E07B680C4A934201D90123BB60BB68AD
:101700001800FFF7EFFEFFF701FF0200BB689342EE
:1017100003D00F23FB1800221A700F23FB181B782D
:101720001800BD4604B080BD00366E0180B584B09F
:1017300000AF786039600023FB603B685B68013371
:101740001900786800F0D0F8030019003B681B68A6
:101750009B0C0F22134002334B43FB60FB681800C5
:10176000BD4604B080BD80B582B000AFFB1D012234
:101770001A70FFF763FE031E02D0FB1D00221A70D1
:10178000FB1D1B781800BD4602B080BD90B585B02A
:1017900000AF786039600F203B1801221A700023D7
:1017A000BB602E4B1A683B681B681B090F210B405E
:1017B0002B49CB5C9A401300BB60BA687B689A42A5
:1017C00006D23C187B681800FFF782FF03002370E5
:1017D0000F23FB181B78012B1AD1FFF721FEC046FF
:1017E000FFF72CFE0300012BFAD13B681B681800A1
:1017F000FFF7ECFD0220FFF7C9FDC046FFF7DAFD59
:101800000300082BFAD13B685B681800FFF7F2FD74
:10181000BA687B689A4207D90F23FC187B681800C6
:10182000FFF756FF030023700F23FB181B78012BD3
:101830000CD13B681B681B090F221340084AD35C7C
:101840001A007B68D3401800FFF79EFE0F23FB1899
:101850001B781800BD4605B090BDC04600000020B2
:10186000241C000880B500AFC046BD4680BD80B5D1
:1018700086B000AFF860B9607A60FA687B68D31808
:101880003B61FB687B6106E0BB68DAB27B691A707A
:101890007B6901337B617A693B699A42F4D3FB68C7
:1018A0001800BD4606B080BD80B584B000AF78603A
:1018B0007B68FB60C0467B685A1C7A601B78002BF3
:1018C000F9D17A68FB68D31A013B1800BD4604B011
:1018D00080BD80B582B000AF0200FB1D1A70C0460B
:1018E000BD4602B080BD0000002243088B4274D385
:1018F00003098B425FD3030A8B4244D3030B8B4211
:1019000028D3030C8B420DD3FF22090212BA030C19
:101910008B4202D31212090265D0030B8B4219D3FA
:1019200000E0090AC30B8B4201D3CB03C01A52411A
:10193000830B8B4201D38B03C01A5241430B8B4262
:1019400001D34B03C01A5241030B8B4201D30B034B
:10195000C01A5241C30A8B4201D3CB02C01A524172
:10196000830A8B4201D38B02C01A5241430A8B4235
:1019700001D34B02C01A5241030A8B4201D30B021E
:10198000C01A5241CDD2C3098B4201D3CB01C01A38
:10199000524183098B4201D38B01C01A5241430942
:1019A0008B4201D34B01C01A524103098B4201D330
:1019B0000B01C01A5241C3088B4201D3CB00C01A9D
:1019C000524183088B4201D38B00C01A5241430815
:1019D0008B4201D34B00C01A5241411A00D201463A
:1019E000524110467047FFE701B5002000F0F0F8C3
:1019F00002BDC0460029F7D076E7704703460B4387
:101A00007FD4002243088B4274D303098B425FD3F7
:101A1000030A8B4244D3030B8B4228D3030C8B4223
:101A20000DD3FF22090212BA030C8B4202D3121209
:101A3000090265D0030B8B4219D300E0090AC30BDE
:101A40008B4201D3CB03C01A5241830B8B4201D38B
:101A50008B03C01A5241430B8B4201D34B03C01A74
:101A60005241030B8B4201D30B03C01A5241C30AEC
:101A70008B4201D3CB02C01A5241830A8B4201D35D
:101A80008B02C01A5241430A8B4201D34B02C01A47
:101A90005241030A8B4201D30B02C01A5241CDD2EC
:101AA000C3098B4201D3CB01C01A524183098B4237
:101AB00001D38B01C01A524143098B4201D34B0120
:101AC000C01A524103098B4201D30B01C01A524183
:101AD000C3088B4201D3CB00C01A524183088B420A
:101AE00001D38B00C01A524143088B4201D34B00F3
:101AF000C01A5241411A00D2014652411046704765
:101B00005DE0CA0F00D04942031000D34042534069
:101B100000229C4603098B422DD3030A8B4212D329
:101B2000FC22890112BA030A8B420CD3890192115B
:101B30008B4208D3890192118B4204D389013AD098
:101B4000921100E08909C3098B4201D3CB01C01A6D
:101B5000524183098B4201D38B01C01A5241430980
:101B60008B4201D34B01C01A524103098B4201D36E
:101B70000B01C01A5241C3088B4201D3CB00C01ADB
:101B8000524183088B4201D38B00C01A5241D9D2F3
:101B900043088B4201D34B00C01A5241411A00D274
:101BA0000146634652415B10104601D34042002B70
:101BB00000D54942704763465B1000D3404201B5EF
:101BC000002000F005F802BD0029F8D016E77047A4
:101BD0007047C0460C488546002103E00B4B5B581C
:101BE000435004310A480B4B42189A42F6D30A4A32
:101BF00002E0002313600432084B9A42F9D3FFF746
:101C0000ADFAFEF70AFBFEE7001000203C1C0008BE
:101C1000000000209400002094000020D403002045
:101C2000FEE70000000000000000000001020304C5
:0C1C300006070809000000000102030480
:101C3C0000127A0000040040002000400028004000
:101C4C00002C004000300040005400400070004068
:101C5C00000001400004014000240140082701401D
:101C6C0008270140002C01400030014000380140A1
:101C7C00004401400048014000580140000002406F
:101C8C00080002401C0002403000024044000240A8
:101C9C00580002400020024000F8FF1F00100240D4
:101CAC0000300240000000480004004800080048D2
:101CBC00000C00480014004800ED00E010E000E0CB
:041CCC0000E100E053
:0400000508001BD5FF
:00000001FF
